:100000000AC023C022C021C020C01FC01EC01DC006
:100010001CC01BC01AC011241FBECFEDCDBF10E005
:10002000A0E6B0E0EEEFF5E003C0C89531960D9282
:10003000A036B107D1F710E0A0E6B0E001C01D92F4
:10004000A936B107E1F751D1D9C2DACFCF93DF9307
:10005000CDB7DEB7E8E3F0E01082E7E3F0E080E15F
:100060008083E2E3F0E01082E1E3F0E08AE0808365
:10007000DF91CF910895CF93DF93CDB7DEB722976D
:100080000FB6F894DEBF0FBECDBFA8E3B0E0E8E343
:10009000F0E080818F7180628C93A7E3B0E0E7E3AA
:1000A000F0E080818F7180628C93E6E3F0E08081E4
:1000B000992780749070009729F081E090E09A83EE
:1000C000898302C01A82198289819A8122960FB689
:1000D000F894DEBF0FBECDBFDF91CF910895CF93CF
:1000E000DF93CDB7DEB722970FB6F894DEBF0FBE11
:1000F000CDBFA8E3B0E0E8E3F0E080818F718064D9
:100100008C93A7E3B0E0E7E3F0E080818F71806437
:100110008C93E6E3F0E0808188232CF481E090E08A
:100120009A83898302C01A82198289819A812296D0
:100130000FB6F894DEBF0FBECDBFDF91CF9108950B
:10014000CF93DF93CDB7DEB722970FB6F894DEBF1B
:100150000FBECDBFA8E3B0E0E8E3F0E08081982FC8
:100160009F7180E8892B8C93A7E3B0E0E7E3F0E090
:100170008081982F9F7180E8892B8C93E6E3F0E0D3
:100180008081992780729070009729F081E090E03B
:100190009A83898302C01A82198289819A81229660
:1001A0000FB6F894DEBF0FBECDBFDF91CF9108959B
:1001B000CF93DF93CDB7DEB722970FB6F894DEBFAB
:1001C0000FBECDBFA8E3B0E0E8E3F0E080818F711F
:1001D00080648C93A7E3B0E0E7E3F0E080818F7167
:1001E00080648C93E6E3F0E08081992780729070C0
:1001F000009729F081E090E09A83898302C01A82F7
:10020000198289819A8122960FB6F894DEBF0FBEBB
:10021000CDBFDF91CF910895CF93DF93CDB7DEB7F8
:1002200022970FB6F894DEBF0FBECDBFA8E3B0E0B3
:10023000E8E3F0E08081982F9F7180E8892B8C9310
:10024000A7E3B0E0E7E3F0E08081982F9F7180E8BA
:10025000892B8C93E6E3F0E080819927807490707D
:10026000009729F081E090E09A83898302C01A8286
:10027000198289819A8122960FB6F894DEBF0FBE4B
:10028000CDBFDF91CF910895CF93DF93CDB7DEB788
:1002900022970FB6F894DEBF0FBECDBFA8E3B0E043
:1002A000E8E3F0E080818F7180628C93A7E3B0E097
:1002B000E7E3F0E080818F7180628C93E6E3F0E009
:1002C000808188232CF481E090E09A83898302C0A6
:1002D0001A82198289819A8122960FB6F894DEBF1C
:1002E0000FBECDBFDF91CF910895CF93DF93CDB7F0
:1002F000DEB768970FB6F894DEBF0FBECDBFA6DE9F
:10030000109268001092670012C08091670090916F
:100310006800F92FE82FE05AFF4F108280916700A4
:100320009091680001969093680080936700809197
:100330006700909168008730910538F300C09BDE1C
:10034000282F3327388F2F8B809161001E8A1D8ABA
:10035000882321F481E090E09E8B8D8B8F89988D8E
:100360002D893E8982239323009751F0A2E3B0E0C8
:10037000E2E3F0E0808188608C9381E0809361000B
:100380007ADE1C8A1B8A882321F481E090E09C8B12
:100390008B8B8091610099272B893C898223932341
:1003A000009751F0A2E3B0E0E2E3F0E0908187EF44
:1003B00089238C931092610092DE882371F1E0E32F
:1003C000F0E08081992788709070009749F0A2E34F
:1003D000B0E0E2E3F0E0908187EF89238C9307C0DF
:1003E000A2E3B0E0E2E3F0E0808188608C9388EEE5
:1003F0009DEF909368008093670009C0809167002B
:1004000090916800019790936800809367008091B5
:10041000670090916800009789F792DE8823D9F1F0
:10042000A8E3B0E0E8E3F0E0808180618C9384EFA2
:1004300091E0909368008093670009C08091670005
:100440009091680001979093680080936700809175
:10045000670090916800009789F7A8E3B0E0E8E3AF
:10046000F0E090818FEE89238C9384EF91E090935C
:1004700068008093670009C08091670090916800D0
:100480000197909368008093670080916700909136
:100490006800009789F78CDE282F33273A8B298B49
:1004A00080916400188A1F86882321F481E090E0FF
:1004B000988B8F8789899A892F85388982239323FE
:1004C000009751F0A2E3B0E0E2E3F0E080818860C1
:1004D0008C9381E0809364006BDE1E861D868823EA
:1004E00021F481E090E09E878D87809164009927B8
:1004F0002D853E8582239323009711F0109264008E
:100500008BDE282F33273C872B87809165001A8646
:100510001986882321F481E090E09A8789878B856A
:100520009C8529853A8582239323009759F0A2E37D
:10053000B0E0E2E3F0E0908187EF89238C9381E0E3
:100540008093650069DE18861F82882321F481E08C
:1005500090E098878F838091650099272F81388557
:1005600082239323009711F0109265008DDE282FCF
:1005700033273E832D83809166001C821B82882353
:1005800021F481E090E09C838B838D819E812B817F
:100590003C81822393230097D9F0E0E3F0E080814F
:1005A000992788709070009749F0A2E3B0E0E2E3E9
:1005B000F0E0908187EF89238C9307C0A2E3B0E03D
:1005C000E2E3F0E0808188608C9381E080936600B4
:1005D0005BDE1A821982882321F481E090E09A83FD
:1005E000898380916600992729813A818223932308
:0E05F000009709F4A4CE10926600A1CEFFCFB2
:00000001FF
